:100000000C945B000C9483000C9483000C9483008C
:100010000C9483000C9483000C9483000C94830054
:100020000C9483000C9483000C9483000C94830044
:100030000C9483000C9483000C9483000C94830034
:100040000C9497020C9483000C9418050C94830074
:100050000C9483000C9483000C9483000C94830014
:100060000C9483000C948300000024272A000025B0
:10007000282B000023262904040404040404040299
:100080000202020202030303030303010204081035
:100090002040800102040810200102040810200002
:1000A0000000070002010000030406000000000039
:1000B00000000000EF0011241FBECFEFD4E0DEBF30
:1000C000CDBF11E0A0E0B1E0E2E8FBE002C00590A6
:1000D0000D92AA30B107D9F711E0AAE0B1E001C052
:1000E0001D92AA39B107E1F710E0C6EBD0E004C0D9
:1000F0002297FE010E94BB05C43BD107C9F70E94AD
:10010000E8000C94BF050C9400000F931F930CE0C3
:1001100011E0BC01C8010E945F0220E030E040E233
:1001200050E060E070E0C8010E9477021F910F91DB
:1001300008951F938CE091E00E940001882359F1FB
:100140008CE091E00E94FD008237910521F510E0DE
:10015000812F0E94770390930B0180930A010E94E4
:1001600085001F5F1630A1F712E0812F0E94520414
:1001700090930B0180930A010E9485001F5F1E303F
:10018000A1F78CE091E00E94300165E070E080E032
:1001900090E00E9402031F91089540E052EC61E05C
:1001A00070E08CE091E00E94030161E08DE00E942C
:1001B000070468E572E080E090E00E94020360E0DE
:1001C0008DE00E94070460E08DE00E94E90308953D
:1001D0000E943A030E94CD000E949900FDCF86E064
:1001E00091E090930D0180930C010895862F0E9459
:1001F000D70408950E940F0508950E94F004089501
:100200000E94DF040895CB01BA010E949E04089564
:10021000DC01ED91FC910190F081E02D09950895AC
:10022000DC01ED91FC910190F081E02D099508959C
:100230000F931F93CF93DF938C01EB0109C021969D
:10024000D801ED91FC910190F081E02DC801099554
:1002500068816623A1F7DF91CF911F910F910895D7
:100260000F931F938C01DC01ED91FC910190F081C3
:10027000E02D6DE00995D801ED91FC910190F081A0
:10028000E02D6AE0C80109951F910F9108950F9321
:100290001F938C01DC01ED91FC910190F081E02D28
:1002A0000995C8010E9430011F910F9108950F9385
:1002B0001F938C010E941801C8010E9430011F91F8
:1002C0000F9108950F931F938C01DC01ED91FC9128
:1002D0000190F081E02D0995C8010E9430011F9125
:1002E0000F9108952F923F924F925F926F927F925B
:1002F0008F929F92AF92BF92CF92DF92EF92FF9236
:100300000F931F93DF93CF93CDB7DEB7A0970FB6B0
:10031000F894DEBF0FBECDBF1C016A017B01411501
:1003200051056105710549F4DC01ED91FC910190E5
:10033000F081E02D60E3099554C08824992454018C
:10034000422E55246624772401E010E00C0F1D1F77
:10035000080D191DC701B601A30192010E9468058D
:10036000F80160830894811C911CA11CB11CC70179
:10037000B601A30192010E946805C901DA016C016E
:100380007D01C114D104E104F104F1F681E0E82E0D
:10039000F12CEC0EFD1EE80CF91C3E010894611CCA
:1003A000711CD501C4010197A109B1096C01C818DC
:1003B000D90814C0F601EE0DFF1D60816A3010F4FB
:1003C000605D01C0695CD101ED91FC910190F0810B
:1003D000E02DC10109950894E108F1086E147F042D
:1003E00049F7A0960FB6F894DEBF0FBECDBFCF91F0
:1003F000DF911F910F91FF90EF90DF90CF90BF9012
:10040000AF909F908F907F906F905F904F903F90B4
:100410002F9008952AE00E94720108950F931F9370
:100420008C010E940A02C8010E9430011F910F91A5
:100430000895AB0160E070E00E940A0208950F93F6
:100440001F938C01AB0160E070E00E940A02C801BA
:100450000E9430011F910F910895EF92FF920F9328
:100460001F93CF93DF93EC017A018B0177FF0FC0CD
:10047000E881F9810190F081E02D6DE209951095F8
:100480000095F094E094E11CF11C011D111D2AE07F
:10049000B801A701CE010E947201DF91CF911F9197
:1004A0000F91FF90EF9008950F931F938C010E947E
:1004B0002D02C8010E9430011F910F910895AB01D8
:1004C000662757FD6095762F0E942D0208950F93A1
:1004D0001F938C01AB01662757FD6095762F0E9414
:1004E0002D02C8010E9430011F910F910895DC0177
:1004F0002115310541F4ED91FC910190F081E02D41
:10050000642F099508952A30310519F40E942D02AF
:1005100008950E94720108950F931F938C010E9409
:100520007702C8010E9430011F910F9108951F9218
:100530000F920FB60F9211242F938F939F93AF9327
:10054000BF9380910E0190910F01A0911001B09185
:1005500011018050904CAF4FBF4F80930E0190938C
:100560000F01A0931001B093110127C080910E01DB
:1005700090910F01A0911001B091110180589E43FC
:10058000A040B04080930E0190930F01A093100102
:10059000B09311018091120190911301A091140167
:1005A000B09115010196A11DB11D80931201909388
:1005B0001301A0931401B093150180910E01909145
:1005C0000F01A0911001B091110181589E43A040EC
:1005D000B04060F6BF91AF919F918F912F910F9096
:1005E0000FBE0F901F9018958FB7F89420911201AD
:1005F0003091130140911401509115018FBFB90141
:10060000CA010895EF92FF920F931F937B018C0113
:100610008FB7F89440911201509113016091140129
:10062000709115018FBF2FB7F894809112019091AE
:100630001301A0911401B09115012FBF841B950BDC
:10064000A60BB70B8E159F05A007B10760F31F918E
:100650000F91FF90EF900895019759F0FC01EE0F74
:10066000FF1FEE0FFF1F32978FB7F8943197F1F706
:100670008FBF0895789484B5826084BD84B581600D
:1006800084BD85B5826085BD85B5816085BDEEE69A
:10069000F0E0808181608083E1E8F0E08081826029
:1006A0008083808181608083E0E8F0E080818160E8
:1006B0008083E1EBF0E0808184608083E0EBF0E018
:1006C000808181608083EAE7F0E0808184608083BC
:1006D0008081826080838081816080838081806866
:1006E00080831092C10008958093080108958F704F
:1006F000909108019295990F990F907C982B909367
:100700007C0080917A00806480937A0080917A00E6
:1007100086FDFCCF2091780040917900942F80E0F5
:1007200030E0282B392BC90108951F93CF93DF9315
:10073000182FEB0161E00E94E903E12FF0E0E156A0
:10074000FF4F8491833051F48091800080688093C2
:100750008000D0938900C093880037C0843051F462
:1007600080918000806280938000D0938B00C09342
:100770008A002BC0813029F484B5806884BDC7BD50
:1007800024C0823029F484B5806284BDC8BD1DC0F8
:10079000863041F48091B00080688093B000C093AF
:1007A000B30013C0873041F48091B0008062809321
:1007B000B000C093B40009C0C038D10514F460E0A3
:1007C00001C061E0812F0E940704DF91CF911F914A
:1007D0000895282F30E0C90185579F4FFC0194915F
:1007E00029583F4FF9018491882381F0E82FF0E0E8
:1007F000E859FF4FE491F0E0662329F48081909559
:100800008923808308958081892B80830895482FD0
:1008100050E0CA0181569F4FFC012491CA018557BF
:100820009F4FFC01949149585F4FFA013491332353
:10083000C1F1222331F1233021F4809180008F77A0
:1008400005C0243031F4809180008F7D809380003A
:1008500018C0213019F484B58F7704C0223021F4F8
:1008600084B58F7D84BD0DC0263021F48091B00009
:100870008F7705C0273029F48091B0008F7D809359
:10088000B000E32FF0E0E359FF4FE491F0E066237E
:1008900029F4808190958923808308958081892B14
:1008A00080830895482F50E0CA0181569F4FFC0174
:1008B0002491CA0185579F4FFC01949149585F4F7D
:1008C000FA013491332319F420E030E035C02223BB
:1008D00031F1233021F4809180008F7705C02430DE
:1008E00031F4809180008F7D8093800018C021308A
:1008F00019F484B58F7704C0223021F484B58F7D3C
:1009000084BD0DC0263021F48091B0008F7705C0E2
:10091000273029F48091B0008F7D8093B000E32FC1
:10092000F0E0EE58FF4FE491F0E0808120E030E00D
:10093000892311F021E030E0C9010895EF92FF9280
:100940000F931F937B018C0122E030E040E050E0E8
:100950000E948A05205C3D4B404F5F4FCA01B901A0
:10096000A80197010E948A05C901DA010197A1092E
:10097000B109292F3A2F4B2F552747FD5A9501963C
:10098000A11DB11D2093C50081508093C400E1ECEE
:10099000F0E08081806180838081886080838081B5
:1009A000806880831F910F91FF90EF900895982F9A
:1009B0008091C00085FFFCCF9093C6000895809180
:1009C00016019091170180589F4F20911801309186
:1009D0001901821B930B60E870E00E945505089591
:1009E00040911801509119018091160190911701C1
:1009F0008417950719F42FEF3FEF0FC0FA01E65E59
:100A0000FE4F2081CA01019660E870E00E94550502
:100A1000909319018093180130E0C90108958091E5
:100A20001801909119019093170180931601089570
:100A30001F920F920FB60F9211242F933F934F9353
:100A40005F936F937F938F939F93AF93BF93EF9336
:100A5000FF934091C600E0911601F0911701CF017C
:100A6000019660E870E00E9455059C018091180194
:100A7000909119012817390739F0E65EFE4F40833F
:100A80003093170120931601FF91EF91BF91AF9121
:100A90009F918F917F916F915F914F913F912F9196
:100AA0000F900FBE0F901F90189597FB092E0726E9
:100AB0000AD077FD04D049D006D000201AF47095F2
:100AC00061957F4F0895F6F7909581959F4F089512
:100AD000A1E21A2EAA1BBB1BFD010DC0AA1FBB1F42
:100AE000EE1FFF1FA217B307E407F50720F0A21BB4
:100AF000B30BE40BF50B661F771F881F991F1A9421
:100B000069F760957095809590959B01AC01BD014A
:100B1000CF01089597FB092E05260ED057FD04D06E
:100B2000D7DF0AD0001C38F45095409530952195B8
:100B30003F4F4F4F5F4F0895F6F790958095709512
:100B400061957F4F8F4F9F4F0895AA1BBB1B51E1AB
:100B500007C0AA1FBB1FA617B70710F0A61BB70B2D
:100B6000881F991F5A95A9F780959095BC01CD01D2
:100B70000895EE0FFF1F0590F491E02D0994F8946D
:020B8000FFCFA5
:0A0B82000D0000000000F600010065
:00000001FF
